:1000000012C02CC02BC02AC029C028C03DC026C0A9
:1000100025C024C023C022C021C020C01FC01EC0D4
:100020001DC01CC01BC011241FBECFE5D4E0DEBF25
:10003000CDBF10E0A0E6B0E0EAE7F6E002C0059030
:100040000D92A23FB107D9F710E0A2EFB0E001C0D6
:100050001D92A73FB107E1F757D00EC3D1CF9CE166
:10006000899FC0011124382F882349F020E0E0E067
:10007000F0E0CF010197F1F72F5F3217D1F7089524
:10008000A89A0895A89808951F920F920FB60F92FC
:1000900011242F938F939F938091F2009091F300FE
:1000A00001969093F3008093F2008091F20090917A
:1000B000F300885E934001F58091F40081508093B5
:1000C000F4001092F3001092F2008091F4008F3F40
:1000D00099F48091F50081508093F5009BE3909313
:1000E000F4008091F5008F3F39F48091F600815043
:1000F0008093F6009093F5009F918F912F910F9030
:100100000FBE0F901F901895EF92FF920F931F93C1
:10011000CF93DF93A09AB6DF88B3876088BB80E077
:100120005CD260E081E0B5D18BE08EBD8AEF90E0DB
:100130009BBD8ABD89B7806189BF789460E081E00A
:10014000A8D180E690E0CCD161E080E039D281E7AF
:1001500090E0C6D184E083DF60E081E09AD182E85C
:1001600090E0BED161E080E02BD283E990E0B8D18D
:1001700006B3FF24EE2411E0402F552786B39927BC
:10018000877090709A012770307082179307B1F3CF
:10019000B29906C042FF04C01F5F133009F4C8C003
:1001A000B1990BC041FF09C0113009F4C3C012302E
:1001B00009F4C7C0112309F4D0C0B0994FC040FF63
:1001C0004DC0113009F4AAC0123009F472C01123D5
:1001D00009F4C3C0CF2DDD27C7FDD09506B360E07D
:1001E00081E057D182E890E07BD161E080E0E8D106
:1001F00080EA90E075D160E08BE0E2D162E070E0EF
:10020000CE017DD160E08EE0DBD162E070E08E2D2A
:10021000992787FD909573D1113009F478C0123079
:1002200009F46EC080E090E0FC013197F1F7FC0129
:100230003197F1F7FC013197F1F7FC013197F1F7B4
:10024000FC013197F1F7FC013197F1F7FC0131978F
:10025000F1F70197F1F7402F552790CF06B360E0F3
:1002600081E017D182E890E03BD161E080E0A8D145
:1002700080EA90E035D160E08BE0A2D162E070E0EE
:100280008F2D992787FD90953AD160E08EE098D127
:1002900062E070E08E2D992787FD909530D1112373
:1002A00009F0BACF61E080E08BD18BEA90E018D101
:1002B000B9CFEA948FEFE81609F44AC0CE2DDD27B6
:1002C000C7FDD09506B360E081E0E3D082E890E01E
:1002D00007D161E080E074D180EA90E001D160E074
:1002E0008BE06ED162E070E08F2D992787FD9095AD
:1002F00006D160E08EE064D162E070E0CE01FFD014
:1003000061E08EE05DD18DEA90E0EAD08BCF61E0D4
:100310008BE056D18DEA90E0E3D084CFFA948FEF52
:10032000F81609F057CF93E6F92EC3E6D0E056CF82
:1003300010E036CFF39484E6F81609F03ECFFF24A0
:100340003CCFE3948CE3E81609F037CFEE2435CFA9
:100350008BE3E82ECBE3D0E0B5CF92DEF092F6004F
:10036000E092F5001092F40060E081E092D08FEA14
:1003700090E0B6D0C0E0D0E00CC0CE010197F1F71C
:10038000CE010197F1F7CE010197F1F7CE01019768
:10039000F1F761E084E014D18091F60062E070E052
:1003A000992787FD9095ABD08FEB90E099D061E0D5
:1003B00087E006D18091F50062E070E0992787FD23
:1003C00090959DD08FEB90E08BD061E08AE0F8D0E3
:1003D0008091F40062E070E0992787FD90958FD0BE
:1003E0008091F600882349F68091F500882309F072
:1003F000C4CF8091F400882309F0BFCF43DE60E0D2
:1004000081E047D081EC90E06BD061E080E0D8D013
:1004100081ED90E065D081E022DE61E080E0D0D027
:1004200081EE90E05DD081E01ADE86B39927809559
:10043000909587709070892B41F36CCE81B3807F4B
:1004400081BB959A969882E08A95F1F722E035E093
:10045000949A822F8A95F1F780B38295807F922FAC
:100460009A95F1F79498932F9A95F1F7949A922F81
:100470009A95F1F790B3922F9A95F1F79498932F5C
:100480009A95F1F787FDE4CF959881B38F6081BB92
:100490000895282F662311F4969801C0969A82E059
:1004A0008A95F1F7949A82B3807F922F92959F70EC
:1004B000892B82BB95E0892F8A95F1F79498892F33
:1004C0008A95F1F7949A82B3807F2F70822B82BB3A
:1004D000892F8A95F1F794989A95F1F7AFDF0895EF
:1004E000CF93DF93EC018881882331F061E0D1DF85
:1004F000219688818823D1F7DF91CF910895EF92DB
:10050000FF920F931F93CF93DF93CDB7DEB725975D
:100510000FB6F894DEBF0FBECDBF9C018B017E01EC
:100520000894E11CF11C85E0F70111928A95E9F726
:100530002115310579F0FE013596C9016AE070E0B8
:1005400074D080833197C9016AE070E06ED09B015E
:10055000672B99F7FFEF0F3F1F07B1F085E090E0A1
:10056000801B910B85309105F4F48C01E00EF11E97
:10057000F70181917F0161E0805D8BDF0F5F1F4F8D
:1005800005301105ACF30FC08981882349F4F701C8
:10059000818131968823E1F3CF018E199F09E2CF43
:1005A00000E010E0E3CF25960FB6F894DEBF0FBE53
:1005B000CDBFDF91CF911F910F91FF90EF900895E4
:1005C000883228F4662321F460E0806862DF0895B1
:1005D000806460E080685DDFFACF1F93182F80E0B1
:1005E00090E00197F1F781B38F6081BB8C9A8E9A6E
:1005F0008D9A82B3807F82BB94989598969881E07B
:100600008A95F1F7949A919A85E0982F9A95F1F747
:1006100094988A95F1F712DF60E0812F8C6039DFC2
:1006200060E088E236DF1F91089597FB092E0726C8
:100630000AD077FD04D00CD006D000201AF47095B3
:1006400061957F4F0895F6F7909581959F4F089596
:10065000AA1BBB1B51E107C0AA1FBB1FA617B707E8
:1006600010F0A61BB70B881F991F5A95A9F7809504
:0A0670009095BC01CD010895FFCF65
:10067A002020202057656C636F6D65202020202084
:10068A000020202052656C61792054696D657220C2
:10069A0020005365742054696D65202D2030303A4E
:1006AA0030300020537461727420202020205E00B4
:1006BA0020537461727420202020003E005E0020C6
:1006CA0020506F776572204F666620496E20003A87
:1006DA00004C6F6164205475726E6564204F6666C3
:1006EA00002A507265737320416E79204B65792A0E
:1006FA000020202020202020202020202020202010
:02070A002000CD
:00000001FF
